:100000000EC228C227C226C225C224C223C222C2CF
:1000100021C220C21FC21EC21DC21CC21BC21AC2E4
:1000200019C20000000000000000000000000000F5
:1000300000000000FEFE000000000000333300005E
:100040000000000C3C00003C0C0000000000000020
:100050000000008080C0B880C0B83A06033A0603AA
:100060000200304884FE848408100408103F1010F9
:100070000906001818806018060060180601000CB8
:100080000C0000B8C4848444380007081010111212
:100090000C0F00001C7C1C00000000000000000091
:1000A000000000F8040200000000000F1020000013
:1000B0000000000204F8000000000020100F000003
:1000C000000090A0C0F8C0A090000402010F01023F
:1000D0000400808080FC808080800000001F000081
:1000E00000000000000000000000004E2E1E0E0068
:1000F0000000808080808080808000000000000000
:1001000000000000000000000000000E1F1F0E0095
:100110000000000000806018060060180601000062
:100120000000F0080402020408F007081020201064
:100130000807000404FE000000000020203F2020EB
:1001400000001804020202028478203028242221B0
:10015000203018040202828244380C102020202013
:10016000110E0080E0380CFE000007050404243F57
:100170002404FE4222222222428208102020202033
:10018000100FF8844242424284080F1020202020A1
:10019000100F0E02020202C2320E0000003C0300E9
:1001A000000038448282828244380E1120202020B0
:1001B000110E78840202020284F808102121212104
:1001C000100F0038383800000000001C1C1C000014
:1001D00000000038383800000000004E2E1E0000DD
:1001E0000000008040201008040000000102040804
:1001F000100030303030303030300606060606064B
:1002000006060004081020408000001008040201C7
:1002100000003804020282824438000000270000F7
:1002200000000000000000000000000000000000CE
:1002300000000000E21E12E00000203F2101012129
:100240003F2002FE828282824438203F20202020EC
:10025000110EF80402020202040E0F1020202020CA
:10026000103802FE0202020204F8203F2020202063
:10027000100F02FE828282C2020E203F2020202127
:10028000203802FE828282C2020E203F200000013E
:100290000000F80402020202040E0F1020232121A4
:1002A0001F3F02FE82808082FE02203F200000204D
:1002B0003F20020202FE020202002020203F2020F6
:1002C0002000000000000002FE02021E222020206A
:1002D0001F0002FEC220100A0602203F200106284D
:1002E000302002FE020000000000203F20202020DD
:1002F000203002FE3EF000F03EFE203F00071E07C9
:10030000003F02FE1EF00000FE02203F00010F38F9
:100310003F20F8040202020204F80F1020202020DF
:10032000100F02FE82828282827C203F2000000029
:100330000000F8040202020204F80F1020262E3CEE
:10034000182F02FE82828282827C203F2003062CAC
:100350003020384482828282020C18202020202003
:10036000110E0E0202FE0202020E0000203F2000CB
:10037000000002FE02000002FE02001F20202020DA
:100380001F00023EC20000E21E02000027382700C4
:10039000000002FE00C078C000FE203F0E030003F4
:1003A0000E3F020E728080720E0220382601012656
:1003B0003820020E728080720E020000203F3F2023
:1003C00000000402020282E23A0E30382C2721207B
:1003D000201000FE020202020000003F2020202028
:1003E00000000618608000000000000000010618F0
:1003F00060000002020202FE000000202020203FD8
:100400000000AE2000B0C8001040813FA1A6A83F68
:10041000A4D300D5F0D922DA12DB208D14AF112439
:100420001FBECFE5D2E0DEBFCDBF10E0A0E6B0E05A
:10043000EAE0FDE002C005900D92AC3DB107D9F7AE
:1004400010E0ACEDB0E001C01D92AA3EB107E1F7AB
:1004500001D359C4D5CDDA9AD99ADA98D9980895A2
:10046000D998DA98D99ADA98089598E087FF02C067
:10047000DA9A01C0DA98D99AD998915011F0880F78
:10048000F5CFDA9AD99AD99808951F93182FE3DFF8
:1004900088E7EBDF80E0E9DF812FE7DFE1DF1F9115
:1004A00008951F93DF93CF930F92CDB7DEB7182F28
:1004B0006983D1DF88E7D9DF80E0D7DF812FD5DFFF
:1004C0006981862FD2DFCCDF0F90CF91DF911F9112
:1004D00008951F93182FBFDF88E7C7DF80E4C5DFCB
:1004E000812FC3DFBDDF1F910895CF93DF938AB3C0
:1004F00086608ABBC0E0D0E0FE01EE5FFB4F8491D6
:10050000C4DF2196CC31D105B9F7DF91CF910895A1
:100510001F93182F862F8055B8DF812F82958F70FB
:10052000612F6F708061BDDF1F9108950F931F933E
:10053000DF93CF930F92CDB7DEB7182F80EBA5DFF7
:1005400080E161E0AEDF87DF88E78FDF80E48DDF69
:1005500009E009C0812F998388DF99819F5F9038D6
:10056000C9F7015011F090E0F5CF7ADF0F90CF91ED
:10057000DF911F910F9108955F926F927F928F92FA
:100580009F92AF92BF92CF92DF92EF92FF920F9322
:100590001F93CF93DF935C01962E742EC0E0D0E0C2
:1005A0008824682D670D892DB3DF552438C053DFAB
:1005B00088E75BDF80E459DF062D10E00052104031
:1005C00084E0000F111F8A95E1F70C0F1D1FEE2428
:1005D000FF24F701E00FF11FEE5DFF4F849145DF2F
:1005E000F60180818E3219F4FE2DF43038F408942F
:1005F000E11CF11C88E0E816F10459F7E62DED3412
:1006000011F0E73531F4882011F482E001C080E276
:100610002CDF80E02ADF80E028DF22DF53946501B1
:10062000C50CD11CF6016080662009F0C0CF839410
:100630002896F82DF23009F0B4CFDF91CF911F91B9
:100640000F91FF90EF90DF90CF90BF90AF909F9071
:100650008F907F906F905F90089586B1856886B97E
:10066000089587B9369A3699FECF24B135B1C901BC
:100670000895EF92FF920F931F93CF93DF9383E040
:1006800090E0EFDFC9E1D0E0EE24FF24870183E0B2
:1006900090E0E7DF8050924097FF03C090958195EE
:1006A0009F4FAA2797FDA095BA2FE816F9060A07CB
:1006B0001B0714F47C018D0180EE90E00197F1F7A7
:1006C00000C00000219719F72091D7003091D80081
:1006D000442737FD4095542FC801B7016CD22091B3
:1006E000E6003091E7003093E9002093E800209184
:1006F000E4003091E5003093E7002093E60028EE17
:1007000033E040E050E083D22093E4003093E500F2
:10071000C901DF91CF911F910F91FF90EF90089544
:1007200064E670E061D2262F205D2093DC006AE051
:1007300070E05AD2605D6093DD009EE29093DE002F
:10074000805D8093DF0081E48093E0001092E100FF
:10075000203319F480E28093DC008CED90E06EE1B0
:1007600042E00ADF8091D9009091DA002091E40004
:100770003091E50082179307B4F42091E6003091A0
:10078000E700821793077CF42091E8003091E9009C
:100790008217930744F480E690E061E044E0ECDEE9
:1007A00021E030E002C020E030E0C9010895482F88
:1007B0008091D9009091DA0064E670E015D2262F7E
:1007C000205D2093DC006AE070E00ED2605D6093F3
:1007D000DD009EE29093DE00805D8093DF0081E487
:1007E0008093E0001092E100203319F480E28093BE
:1007F000DC008CED90E06EE1BFDE089564E670E011
:10080000F3D1605D6093DC006AE070E0EDD1605D83
:100810006093DD00805D8093DE001092DF008CED40
:1008200090E0089581E090E043D29C019093D8003D
:100830008093D700843691053CF488EE91E0909344
:10084000D8008093D700089583E02538380734F026
:1008500084E893E09093D8008093D7000895CF93D5
:10086000DF9380E063DE8EE690E065E041E084DEC9
:100870008AE790E065E046E07FDE8091D7009091C6
:10088000D800BCDF69E143E077DE8FE996E8A1E0BC
:1008900081509040A040E1F700C00000C0E0D0E0EF
:1008A0008091D7009091D800A9DF69E143E064DE30
:1008B000AFE4B3EC1197F1F700C00000B19B02C0A8
:1008C00021960FC08091D7009091D800B3E0843872
:1008D0009B072CF401969093D8008093D700C0E03A
:1008E000D0E0B0990DC08091D7009091D8008536A6
:1008F0009105A4F201979093D8008093D700CECFB2
:10090000C431D1056CF26091D7007091D80081E0BC
:1009100090E0D3D187DF86E890E065E046E02CDE0A
:100920008FE79AE1A6E081509040A040E1F700C037
:100930000000DF91CF9108958AE090E0B9D19C0149
:100940009093DA008093D900181619063CF08EE1D6
:1009500090E09093DA008093D900089581E02D32E1
:10096000380734F08CE291E09093DA008093D9005C
:100970000895CF93DF9380E0D9DD82E990E065E0D0
:1009800041E0FADD8AE790E065E046E0F5DD83E0EE
:1009900090E00DDF8FE996E8A1E081509040A04003
:1009A000E1F700C00000C0E0D0E083E090E0FFDEAF
:1009B000AFE4B3EC1197F1F700C00000B19B02C0A7
:1009C00021960FC08091D9009091DA00B1E08C326D
:1009D0009B072CF401969093DA008093D900C0E035
:1009E000D0E0B0990DC08091D9009091DA008230AA
:1009F0009105CCF201979093DA008093D900D3CF80
:100A0000C431D10594F26091D9007091DA008AE086
:100A100090E053D191DF86E890E065E046E0ACDD00
:100A20008FE79AE1A6E081509040A040E1F700C036
:100A30000000DF91CF910895009719F4D898DF9ABC
:100A40000895D89ADF980895009711F4C2980895F0
:100A5000C29A0895CF93DF9387EA91E60197F1F761
:100A600000C0000087E08ABB84E087BB80E090E0A4
:100A7000E3DF8FE39DE0A3E081509040A040E1F7E9
:100A800000C0000081E090E0DFDF2FDDA7EAB1E6E3
:100A90001197F1F700C0000080E090E0D5DF8FEF04
:100AA00045DD8FE39DE0A3E081509040A040E1F759
:100AB00000C00000D2DD80E039DDB4DE8FE996E8C9
:100AC000A1E081509040A040E1F700C0000081E02B
:100AD00090E0BADF8EE990E065E040E04DDD83EA2A
:100AE00090E06FE042E048DD8BEA90E069E144E0AD
:100AF00043DD85EB90E063E246E03EDD8FE39EE779
:100B0000A5E081509040A040E1F700C00000B19BFB
:100B100001C0B09BA4DE80E090E096DFAFE4B3ECD0
:100B20001197F1F700C0000007DFA3DD81E090E03E
:100B300083DFC0E0D0E0209789F480E0F7DC8BEB26
:100B400090E062E040E018DD89EC90E062E044E093
:100B500013DD86E090E02BDEC9E1D0E081E090E09B
:100B600073DF87DDDDDD181619062CF480E090E0D8
:100B700063DF94E016C0B19B04C0B09B02C0219714
:100B800003C0F7DEC0E0D0E080E090E05DDF8FE6FC
:100B900091E1A1E081509040A040E1F700C0000049
:100BA000CACF88B3892788BBA3EDB0E31197F1F7CB
:100BB00000C00000F6CFFF27EE27BB27AA2760FF63
:100BC00004C0A20FB31FE41FF51F220F331F441FE1
:100BD000551F969587957795679589F700977607BE
:100BE00071F7CF01BD01089597FB092E07260AD0A2
:100BF00077FD04D027D006D000201AF470956195B7
:100C00007F4F0895F6F7909581959F4F089597FB34
:100C1000092E05260ED057FD04D028D00AD0001C7E
:100C200038F450954095309521953F4F4F4F5F4F89
:100C30000895F6F790958095709561957F4F8F4F49
:100C40009F4F0895AA1BBB1B51E107C0AA1FBB1FE2
:100C5000A617B70710F0A61BB70B881F991F5A9548
:100C6000A9F780959095BC01CD010895A1E21A2EB7
:100C7000AA1BBB1BFD010DC0AA1FBB1FEE1FFF1F40
:100C8000A217B307E407F50720F0A21BB30BE40B90
:100C9000F50B661F771F881F991F1A9469F76095D7
:100CA0007095809590959B01AC01BD01CF01089591
:100CB000A8E1B0E042E050E006C00196272F12D034
:100CC00010C0DC01CB01FC01E199FECF06C0FFBBE7
:100CD000EEBBE09A31960DB20D9241505040B8F7FC
:100CE0000895262FE199FECF9FBB8EBBE09A019716
:100CF0000DB2021639F01CBA2DBB0FB6F894E29A69
:0A0D0000E19A0FBE0895F894FFCFAA
:100D0A002020545249505045442020202000534569
:100D1A005420414353204D463A00505245535320E4
:100D2A0055502F444E002020205341564544202040
:100D3A002000545249502056414C55453A005341DF
:100D4A0046450043555252454E54004150504C4975
:100D5A00414E4345004755415244005245414420C3
:100D6A0043555252454E543A005452495020435525
:0C0D7A005252454E543A00E8011E0000A1
:00000001FF
